:04000000B601DD293F
:10000800B616B61EB612B6190D28B6154620031830
:1000180034280830A3005A20A20DA30B0F28B61EBF
:100028003F2064206020B61A3420392022080310AB
:10003800D829B616B61EB61236192728FE39B700C3
:1000480036150310D829361A2F28A600361646204A
:100058000318342826084D2003183428B61ED8293A
:100068003F20642036113612B6113A088400380849
:100078008417800445283A088400380980058417C5
:1000880080050800392064203F2060203708B61911
:100098000138A2000830A300A20D03183920031C60
:1000A8003F2064206020A30B5028392064203A08A0
:1000B800840038080005FF3E3B08840039094228BF
:1000C8003B08840039083C280408A6003A08840044
:1000D8008030B7050830A70003100318B70A82203C
:1000E800A60CA70B71280000AB1A370C8220DB2165
:1000F800031482202F08A3002E0841298413AB1F64
:100108009128000838042B1F38068000841700083F
:100118003804031C380680009C2800083804031C97
:1001280038062B1B380680008417380980059C2860
:100138002B081F39003EA1002A08083E0318A10A0F
:1001480000004E29B71329080319B7170430A8006F
:10015800250EB3202508B320240EB32024080F3918
:10016800F63E0318073E0A3ED628B7132908031996
:10017800B7170530A8002730A3001030CF20033070
:10018800A300E830CF20A3016430CF20A3010A30B8
:10019800CF202408D628A2002508A1002408A00002
:1001A800A1212008A000A8030319B71329080319DF
:1001B800E0282802031808002008031DB713B71BFE
:1001C8000800303ED3290830A600A7003B08840069
:1001D800390837193421371D36213A088400380880
:1001E8003921A001A10126080319D829B7182B2104
:1001F8003A08840000083805FF3EA00DA10DB71C81
:100208002B21A60BFA282708371862292008D82995
:100218000830A6003B088400390837193421371DF7
:1002280036213A08840038093D2126080319D829BF
:10023800371862213A088400A10CA00C0008380481
:10024800031C380680002B21A60B1E29D8293B0841
:100258008400390880060000312932298006080008
:1002680080043C29FF3A80053D2984178004D82959
:10027800FF3A84178005D829A301A200FF30A207FE
:10028800031CA307031CD8290330A100E4304E2126
:100298004229A101F63EA000A109031C5929FE30FC
:1002A8000000A00703185429A0076400A10F5329D0
:1002B800000020185F29201861290800A201A30165
:1002C8006929A10CA00CA20DA30DFF3E03186529F6
:1002D8002308A1002208A000D829A20002307F2903
:1002E800A20003307F29A20001307F29A200063036
:1002F8007F29A2000530A80023082102031D8629B2
:10030800220820020430031801300319023028059E
:10031800031DFF30D8290404031DFF30D829A2008B
:100328002008A6002408A0002608A4002108A6008A
:100338002508A1002608A500A329A501A4011030BD
:10034800A600210DA40DA50D2208A4022308031C54
:10035800230FA5020318B7292208A40723080318A6
:10036800230FA5070310A00DA10DA60BA529200892
:10037800D8291030A800A101A001A70CA60C031CC5
:10038800CB292208A00723080318230FA107A10CD3
:10039800A00CA50CA40CA80BC1292408D8298400FA
:1003A80031088A0030088200831303138312640023
:1003B8000800831607309F00AA01AB01A801A90114
:1003C8008312DA01DB01D801D901E201E301E0017E
:1003D800E1018316D201D6018613061386129030E6
:1003E8008700D3018312CC01CD018316D801AE0159
:1003F800AF018312C601C701F401F501BC01BD01BB
:100408000130A300F4308A01412186138316861334
:100418008312861283168612831206138316061316
:1004280007308312BA004030B8002030AA00AB0170
:10043800AE01AF0153308A01692074308A01692006
:1004480061308A01692072308A01692074308A011A
:10045800692069308A0169206E308A016920673015
:100468008A0169202E308A0169202E308A0169208C
:100478002E308A0169202E308A0169200A308A01CB
:1004880069200D308A0169208A110A16A32A0714E7
:100498008316FF30D1000A30CF0083128A110A1266
:1004A8000925071032308A01402183164030CE00DA
:1004B8009530D000831283164E08D100073083127E
:1004C800BA002030B8000730BB000830B90001304E
:1004D800B700831651088312A000A1018A010C21DC
:1004E8008316D1010430CF0083128A110A1209251C
:1004F80083165008D10007308312BA002030B800A4
:100508000730BB000830B9000130B7008316510826
:100518008312A000A1018A010C2183160130CD00AD
:1005280083128A110A122523071432308A014021C6
:100538000710640083165908003C8A110A128312B6
:100548000319E92A07148316FF30D10007308312F4
:10055800BA002030B8000730BB000830B9000130BD
:10056800B700831651088312A000A1018A010C214B
:100578008A110A128525071083164130D1000730E9
:100588008312BA002030B8000730BB000830B90029
:100598000130B700831651088312A000A1018A0117
:1005A8000C218316D1010430CF0083128A110A125C
:1005B80009258316FF30D10083128A110A12622599
:1005C8008A110A1285258A019D2A8316FF30D100D7
:1005D80007308312BA004030B8002030AA00AB01BF
:1005E800AE01AF014D308A0169204D308A01692082
:1005F80043308A01692020308A01692049308A0104
:1006080069204E308A01692049308A0169205430B6
:100618008A01692020308A0169204F308A016920C7
:100628004B308A01692021308A0169200A308A0109
:1006380069200D308A016920861683168612831276
:1006480008006400831659084D028A110A128312A1
:1006580003193E2B0730BA001030B8000730BB0032
:100668000830B900B7018A01E7208316D900831240
:100678008A01252B08008617831686138312071410
:100688008316FF30CC0083128A110A1273258A114F
:100698000A128525071083165830C80083123F08B0
:1006A8008316C90083123E088316CA0083124108C4
:1006B8008316CB00831240088316CC0083128A115C
:1006C8000A122F258316FF30CC0083128A110A12D2
:1006D80073258A110A1285258316CD0183128A0192
:1006E80025238316FE30CC0083128A110A12732543
:1006F8004E08BC004F08BD003C08A0003D08A10002
:100708005108A30050088A0177218A110A12031D93
:10071800BB2B0730BA000230B8000730BB000430EA
:10072800B900A0308A011F203D088A011F203C081B
:100738008A011F208A0104208316D1000730831202
:10074800BA002030B8000730BB000830B9000130CB
:10075800B700831651088312A000A1018A010C2159
:10076800BC0A0319BD0A8A110A12031D802B8316BD
:10077800FF30D1000230CF0083128A110A120925F6
:100788008A110A1285250F3083165905DC00831259
:100798008A110A128525640083165908003C8A11BB
:1007A8000A128312031DE82B0730BA001030B80074
:1007B8000730BB000830B900B7018A01E72083166B
:1007C800D90083128A01CF2B8A110A12C3248613F7
:1007D800831686138312080007148316FF30CC0093
:1007E80083128A110A1273258A110A1285250710A5
:1007F80083165130C80083123F088316C90083123C
:100808003E088316CA00831241088316CB00831260
:1008180040088316CC0083128A110A122F258316EA
:10082800FF30CC0083128A110A1273258A110A122A
:1008380085258316CD0183128A0125238316FE3070
:10084800CD0083128A0125234E08CA004F08CB0029
:100858004A08A0004B08A1005108A30050088A01CB
:1008680077218A110A12031D642C0730BA00103050
:10087800B8000730BB000830B900B7018A01E7208B
:100888008316D10007308312BA000230B80007304F
:10089800BB000430B900A0308A011F204B088A0130
:1008A8001F204A088A011F208316510883128A01D3
:1008B8001D20CA0A0319CB0A8A110A12031D2C2CFF
:1008C8008A110A1285258A110A1285258A110A12A7
:1008D800C324080083165030CE0083128A110A12EE
:1008E8008E24080083166030CE0083128A110A1203
:1008F8008E24080083166130CE0083128A110A12F2
:100908008E24080083166630CE0083128A110A12DC
:100918008E24080007148316FF30CC0083128A1136
:100928000A1273258A110A128525071083164E08A4
:10093800C80083123F088316C90083123E08831635
:10094800CA00831241088316CB008312400883161D
:10095800CC0083128A110A122F258316FF30D1008A
:100968000230CF0083128A110A1209258A110A124D
:1009780085258316CD0183128A01252308000714D3
:100988008316FF30D10007308312BA002030B80038
:100998000730BB000830B9000130B7008316510892
:1009A8008312A000A1018A010C218A110A1285254F
:1009B800071083164D30CC0083128A110A12732552
:1009C8008316D1010430CF0083128A110A12092537
:1009D8008316FF30CC0083128A110A127325073060
:1009E800BA001030B8000730BB000830B900B701B2
:1009F80010308A01E8208316A60083122108831686
:100A0800A7002608D8008312080083160130DC00EE
:100A18008312640083165C084F028A110A1283123B
:100A2800031C2E2D0730BA002030B8000730BB0059
:100A38000830B9000130B700831651088312A000AE
:100A4800A1018A010C218316DC0A8A110A12831279
:100A5800031D0D2D08000730BA002030B8000730FC
:100A6800BB000830B9000130B7008316480883126C
:100A7800A000A1018A010C210730BA002030B8007B
:100A88000730BB000830B9000130B70083164908A9
:100A98008312A000A1018A010C210730BA0020307E
:100AA800B8000730BB000830B9000130B700831622
:100AB8004A088312A000A1018A010C210730BA005C
:100AC8002030B8000730BB000830B9000130B7004B
:100AD80083164B088312A000A1018A010C2107305C
:100AE800BA002030B8000730BB000830B900013028
:100AF800B70083164C088312A000A1018A010C21BB
:100B080008000730BA001030B8000730BB000830C2
:100B1800B900B7018A01E7208316D90083120800BB
:100B2800CE010830CF00FF30D0000930D100BE011F
:100B3800BF01C001C1018A01F0230B30BC0008309D
:100B4800BD000730BA000230B8000730BB000430DF
:100B5800B900A0308A011F203D088A011F203C08E7
:100B68008A011F208A010420C4000C30BC00083010
:100B7800BD000730BA000230B8000730BB000430AF
:100B8800B900A0308A011F203D088A011F203C08B7
:100B98008A011F208A010420C5000D30BC000830DE
:100BA800BD000730BA000230B8000730BB0004307F
:100BB800B900A0308A011F203D088A011F203C0887
:100BC8008A011F208A0104208316DA0083120E305E
:100BD800BC000830BD000730BA000230B80007304A
:100BE800BB000430B900A0308A011F203D088A01EB
:100BF8001F203C088A011F208A0104208316AC00AC
:100C080083120F30BC000830BD000730BA00023034
:100C1800B8000730BB000430B900A0308A011F209B
:100C28003D088A011F203C088A011F208A010420F0
:100C38008316AD0083121130BC000830BD000730A8
:100C4800BA000230B8000730BB000430B900A03049
:100C58008A011F203D088A011F203C088A011F20A5
:100C68008A0104208316A40083121230BC000830C5
:100C7800BD000730BA000230B8000730BB000430AE
:100C8800B900A0308A011F203D088A011F203C08B6
:100C98008A011F208A0104208316A50083121630BA
:100CA800BC000830BD000730BA000230B800073079
:100CB800BB000430B900A0308A011F203D088A011A
:100CC8001F203C088A011F208A010420F6001730E3
:100CD800BC000830BD000730BA000230B800073049
:100CE800BB000430B900A0308A011F203D088A01EA
:100CF8001F203C088A011F208A010420F7001330B6
:100D0800BC000830BD000730BA000230B800073018
:100D1800BB000430B900A0308A011F203D088A01B9
:100D28001F203C088A011F208A0104208316B8006E
:100D380083121430BC000830BD000730BA000230FE
:100D4800B8000730BB000430B900A0308A011F206A
:100D58003D088A011F203C088A011F208A010420BF
:100D68008316B900B601B70138088312A0008316AC
:100D780039088312A100A30100308A017D218A115C
:100D88000A12031D2F2F2030BC000830BD00073089
:100D9800BA000230B8000730BB000430B900A030F8
:100DA8008A011F203D088A011F203C088A011F2054
:100DB8008A0104208316B80083122130BC00083051
:100DC800BD000730BA000230B8000730BB0004305D
:100DD800B900A0308A011F203D088A011F203C0865
:100DE8008A011F208A0104208316B9008312223049
:100DF800BC000830BD000730BA000230B800073028
:100E0800BB000430B900A0308A011F203D088A01C8
:100E18001F203C088A011F208A0104208316B6007F
:100E280083122330BC000830BD000730BA000230FE
:100E3800B8000730BB000430B900A0308A011F2079
:100E48003D088A011F203C088A011F208A010420CE
:100E58008316B7008312831624088312A60083160C
:100E680025088312A7002030A200A3018A01BD2112
:100E7800B2002508B3004408B20745080318013E2C
:100E8800B3070130B2020030031C013EB30232083E
:100E9800A0003308A1004408A2004508A3008A0165
:100EA800A1218316A200831221088316A3008312AE
:100EB8000230A600A7017608A2007708A3008A01DD
:100EC800BD21B2002508B30083162C088312B2078F
:100ED80083162D080318013E8312B30732088316C0
:100EE80022078312F80033080318013E83162307EC
:100EF8008312F9007808A6007908A7004408A20020
:100F08004508A3008A01BD21FC002508FD007808DA
:100F1800A6007908A7004408A2004508A3008A0192
:100F2800BD212008FA002108FB007A08D4007B08BC
:100F3800D5007C08D6007D08D700D801D90144081F
:100F4800A6004508A70083162C088312A200831662
:100F58002D088312A3008A01BD21DA002508DB00D1
:100F68007608A6007708A700A2010230A3008A012C
:100F7800BD21E2002508E3007608A6007708A7004F
:100F8800A2010230A3008A01BD212008E000210847
:100F9800E1005A08E2075B080318013EE307640012
:100FA8008A110A12031CDB2FE00A0319E10A7608EA
:100FB800A6007708A700A2010230A3008A01BD217C
:100FC80020088316A800831221088316A90083121B
:100FD8007608A6007708A700A2010230A3008A01BC
:100FE800BD218316AA00831225088316AB0083123D
:100FF80060088316A807831261080318013E831648
:10100800A907831262088316AA07831263080318C4
:10101800013E8316AB0764008A150A128312031C6B
:101028001A288316A80A0319A90A831283163608F0
:101038008312A000831637088312A100A301003091
:101048008A017A218A150A12031D2D288A150A1287
:101058005F28780883163802B20083127908031CC7
:10106800013E83163902B30032088312A0008316AA
:1010780033088312A10083165A088312A200A30121
:101088008A01A1218316B200831221088316B300B6
:1010980032088312A000831633088312A1000F3090
:1010A800A300F5308A0174218A150A12031D5F28EE
:1010B8008A110A161C2B83161030D500831283164A
:1010C8005A088312A600A7014408A2004508A300F5
:1010D8008A01BD21C8002508C9000800CE010230D8
:1010E800CF00FF30D0000330D100831628088312C8
:1010F800BE00831629088312BF0083162A088312AC
:10110800C00083162B088312C1008A01F023073020
:10111800BA000230B8000730BB000430B900A03074
:101128008A011F2002308A011F203F308A011F20B8
:101138008A010420FF000730BA000230B8000730E7
:10114800BB000430B900A0308A011F2002308A0198
:101158001F203E308A011F208A010420FE0007302C
:10116800BA000230B8000730BB000430B900A03024
:101178008A011F2002308A011F203D308A011F206A
:101188008A0104208316A10007308312BA000230B6
:10119800B8000730BB000430B900A0308A011F2016
:1011A80002308A011F203C308A011F208A01042056
:1011B8008316A00007308312BA000230B800073047
:1011C800BB000430B900A0308A011F2002308A0118
:1011D8001F203B308A011F208A0104208316B1009A
:1011E80007308312BA000230B8000730BB00043061
:1011F800B900A0308A011F2002308A011F203A302E
:101208008A011F208A0104208316B00083127E08F9
:101218008316BE0083127F088316BF002008C00013
:101228002108C100831248088316BC0083124908AC
:101238008316BD0083128A150A12402702308316CE
:1012480044078312D200831645080318013E83120F
:10125800D300831630088312A00083163108831246
:10126800A100A30100308A017D218A150A12031DFD
:10127800702983160230B000B10107308312BA001A
:101288000230B8000730BB000430B900A0308A0132
:101298001F2002308A011F203B308A011F2083163D
:1012A800310883128A011D200730BA000230B800C5
:1012B8000730BB000430B900A0308A011F2002307B
:1012C8008A011F203A308A011F20831630088312B2
:1012D8008A011D20C601C7017E08D4007F08D500F9
:1012E800831620088312D600831621088312D7009C
:1012F8007C08D6077D080318013ED70764008A15C5
:101308000A12031C8A29D40A0319D50A831620084D
:101318008312A000831621088312A100A3010030C4
:101328008A017721B2007E08A0007F08A100A301EE
:1013380000308A017721B4003208840034088A0119
:101348008F21B400B5006400340835048A150A12E8
:101358000319CD297E088316BE0083127F088316E1
:10136800BF002008C0002108C10083124808831666
:10137800BC00831249088316BD0083128A150A121D
:101388004027831642088312C60083164308831237
:10139800C7008A150A123E2283162C08831274028B
:1013A800B20083162D08031C013E83127502B30098
:1013B8003208A0003308A1000330A200A3018A016B
:1013C800A12124088316DB005B0883127402B20093
:1013D8007508031CFF3EB3003208A6003308A700B7
:1013E8004408A2004508A3008A01BD21DE002508A3
:1013F800DF0083165B0883127402B2007508031CB1
:10140800FF3EB3003208A6003308A7004408A20034
:101418004508A3008A01BD212008DC002108DD0061
:101428007608A6007708A7004408A2004508A3008C
:101438008A01BD21E6002508E7007608A60077089E
:10144800A7004408A2004508A3008A01BD2120087E
:10145800E4002108E5005E08E6075F080318013E7E
:10146800E70764008A150A12031C3D2AE40A0319D7
:10147800E50A08006400831655080C3C8A150A1210
:101488008312031D732A0310530CEF00520CEE0055
:101498005208EE0753080318013EEF0764008A1547
:1014A8000A12031C5D2A0130EC00ED018A150A12AC
:1014B8005F2AEC01ED015208A6005308A70003308B
:1014C800A200A3018A01BD21B2002508B3000310C0
:1014D800330CEB00320CEA008A150A12902A5208E3
:1014E800A6005308A7000230A200A3018A01BD216B
:1014F800EE002508EF005208A6005308A7000230A6
:10150800A200A3018A01BD212008EC002108ED00FA
:101518006E08EA006F08EB006A08A0006B08A100DB
:10152800A2010630A3008A01A1212408CC002508C5
:10153800CD006C088316BE0083126D088316BF00A9
:1015480083126E088316C00083126F088316C100C9
:10155800831244088316BC00831245088316BD0015
:1015680083128A150A124027831644082C0783120F
:10157800F400831645080318013E2D078312F50071
:101588007408A6007508A7004408A2004508A3002F
:101598008A01BD21DA002508DB007408A600750859
:1015A800A7004408A2004508A3008A01BD2120081D
:1015B800D8002108D9007608A6007708A7004408B3
:1015C800A2004508A3008A01BD21E2002508E30026
:1015D8007608A6007708A7004408A2004508A300DB
:1015E8008A01BD212008E0002108E1005A08E2072D
:1015F8005B080318013EE30764008A150A12031CFE
:10160800082BE00A0319E10A0800CE011030CF00C8
:10161800FF30D0001130D1005C08BE005D08BF006B
:101628005E08C0005F08C1008A01F023CE011230B5
:10163800CF00FF30D0001330D1000030C007023097
:101648000318013EC10764008A150A12031C2F2BD8
:10165800BE0A0319BF0A8A01F023CE011430CF0055
:10166800FF30D0001530D10000305E07C0000430D4
:101678000318013E5F07C10064008A150A12031CA3
:10168800482BBE0A0319BF0A8A01F02308008316F3
:101698005030CE008312BE01BF014208C00043088B
:1016A800C1008A018E2408005608A0005708A1002E
:1016B800FF30A300FF308A017D218A150A12031D1D
:1016C8006D2BD40A0319D50AD601D7018A150A1237
:1016D800702BD60A0319D70A08008316200883122C
:1016E800A000831621088312A100FF30A300FF3059
:1016F8008A017D218A150A12031D8C2BFE0A031903
:10170800FF0A8316A001A10183128A150A12912BE0
:101718008316A00A0319A10A831208000730BA0029
:101728000230B8000730BB000430B900A0308A018D
:101738001F2083162F0883128A011F2083162E0864
:1017480083128A011F208316520883128A011D20E2
:101758008316AE0A0319AF0A8312C60A0319C70A09
:101768008A150A1271234608A0004708A1004908F3
:10177800A30048088A017D218A150A12031D0B2C33
:101788008A150A1257265008A0005108A1001530E2
:10179800A300FF308A017D218A150A12031DD82B68
:1017A80083160130D30083128A150A12D6246400E6
:1017B80083165308013C8A150A128312031D032C51
:1017C8000030DE0706300318013EDF0764008A1583
:1017D8000A12031CF22BDC0A0319DD0A0030E607A3
:1017E80006300318013EE70764008A150A12031C35
:1017F800002CE40A0319E50A8A150A120923D20AF9
:101808000319D30AC601C7018316D30183128316AD
:101818002E088312A00083162F088312A10002301D
:10182800A30000308A017D218A150A12031DBB2CF2
:101838000730BA000230B8000730BB000430B900E6
:10184800A0308A011F2002308A011F203F308A0100
:101858001F207F088A011D200730BA000230B80017
:101868000730BB000430B900A0308A011F200230C5
:101878008A011F203E308A011F207E088A011D2010
:101888000730BA000230B8000730BB000430B90096
:10189800A0308A011F2002308A011F203D308A01B2
:1018A8001F208316210883128A011D200730BA00E1
:1018B8000230B8000730BB000430B900A0308A01FC
:1018C8001F2002308A011F203C308A011F20831606
:1018D800200883128A011D2054087A07BE00550883
:1018E8000318013E7B07BF005608A0005708A10057
:1018F800A2010230A3008A01A1212408B200250810
:10190800B30032085602C0003308031C013E5702D8
:10191800C100CE01CF01FF30D0000130D1008A01D3
:101928003F235608A0005708A100FD30A300FF3050
:101938008A017A218A150A12031DAE2CD40A0319CA
:10194800D50A0030D60702300318013ED7078A159A
:101958000A12B42C0030D60702300318013ED7070C
:101968008316AE01AF0183128A150A12BC2408003F
:10197800CE010230CF00FF30D0000330D1008316F3
:1019880028088312BE00831629088312BF00831615
:101998002A088312C00083162B088312C1008A010B
:1019A8003F2308008A150A123E220730BA00403049
:1019B800B8002030AA00AB01AE01AF0146308A0161
:1019C800692061308A01692074308A0169205330A6
:1019D8008A01692065308A01692063308A0169209B
:1019E8003A308A0169200430A9007408A4007508F7
:1019F800A5006830B000B1018A01A62020308A0114
:101A0800692046308A01692061308A016920743072
:101A18008A01692031308A0169203A308A016920B7
:101A28000430A9005C08A4005D08A5006830B00077
:101A3800B1018A01A6200430A9005E08A4005F084D
:101A4800A5006830B000B1018A01A62020308A01C3
:101A580069204F308A01692066308A016920663022
:101A68008A01692053308A01692065308A0169201A
:101A780074308A0169203A308A0169200430A9004B
:101A88004C08A4004D08A5006830B000B1018A01D7
:101A9800A62020308A01692045308A01692041301A
:101AA8008A01692064308A01692064308A016920CA
:101AB8000430A9004E08A4004F08A5006830B00003
:101AC800B1018A01A6200430A9005008A4005108D9
:101AD800A5006830B000B1018A01A620CE011030FF
:101AE800CF00FF30D0001130D1005C08BE005D0887
:101AF800BF005E08C0005F08C1008A013F23640878
:101B0800BE006508BF006608C0006708C1008A01FA
:101B18003F230730BA004030B8002030AA00AB019C
:101B2800AE01AF0120308A01692046308A01692060
:101B380061308A01692074308A01692032308A0153
:101B480069203A308A0169200430A9003E08A400BF
:101B58003F08A5006830B000B1018A01A620043012
:101B6800A9004008A4004108A5006830B000B101F0
:101B78008A01A6200D308A0169200A308A0169206D
:101B8800CE011230CF00FF30D0001330D1005C08F6
:101B9800BE005D08BF0000305E07C00002300318B9
:101BA800013E5F07C10064008A150A12031CDF2D7D
:101BB800BE0A0319BF0A8A013F236408BE006508EC
:101BC800BF0000306607C00002300318013E6707F7
:101BD800C10064008A150A12031CF52DBE0A0319F8
:101BE800BF0A8A013F23CE011430CF00FF30D00056
:101BF8001530D1005C08BE005D08BF0000305E07EC
:101C0800C00004300318013E5F07C10064008A1554
:101C18000A12031C122EBE0A0319BF0A8A013F23A7
:101C28006408BE006508BF0000306607C0000430C5
:101C38000318013E6707C10064008A150A12031CD5
:101C4800282EBE0A0319BF0A8A013F230800CA01C9
:101C58001030CB004A08A0004B08A1001530A300A3
:101C6800FF308A0177218A150A12031D562E073084
:101C7800BA000230B8000730BB000430B900A03009
:101C88008A011F204B088A011F204A088A011F2049
:101C980000308A011D20CA0A0319CB0A8A150A12C4
:101CA800031D2E2E08005208A6005308A700023074
:101CB800A200A3018A01BD21EA002508EB006A08F9
:101CC800A0006B08A100A2010630A3008A01A1218F
:101CD8002408CC002508CD0000304C07CE00103079
:101CE8000318013E4D07CF0001304E07D0004F08C2
:101CF8000318013ED1005008A0005108A10015307A
:101D0800A300FF308A017D218A150A12031DC62E01
:101D1800013052078316B400831253080318013E9A
:101D28008316B50007308312BA000230B8000730B6
:101D3800BB000430B900A0308A011F204F088A0177
:101D48001F204E088A011F208316340883128A0137
:101D58001D200730BA000230B8000730BB0004303D
:101D6800B900A0308A011F2051088A011F2050089D
:101D78008A011F208316350883128A011D208A15BF
:101D88000A12072F0730BA000230B8000730BB002C
:101D98000430B900A0308A011F204F088A011F2093
:101DA8004E088A011F20FF308A011D200730BA0023
:101DB8000230B8000730BB000430B900A0308A01F7
:101DC8001F2051088A011F2050088A011F20FF3058
:101DD8008A011D205208A0005308A100A301023067
:101DE8008A0171218A150A12031D3F2F4E08A0008F
:101DF8004F08A1001030A30000308A0171218A1514
:101E08000A12031D3F2F0730BA000230B80007300E
:101E1800BB000430B900A0308A011F2002304E02F6
:101E2800B2000030031C013E4F02B30033088A01A0
:101E38001F2032088A011F2052088A011D200730FE
:101E4800BA000230B8000730BB000430B900A03037
:101E58008A011F2002305002B2000030031C013EEC
:101E68005102B30033088A011F2032088A011F205B
:101E780053088A011D20080083163E088312A0001B
:101E880083163F088312A100831640088312A4001A
:101E9800831641088312A50083163D088312A30008
:101EA80083163C0883128A0193218316C400831287
:101EB80021088316C500831224088316C2008312E2
:101EC80025088316C300831208000800CE01CF013D
:101ED800FF30D0000130D100BE01BF01C001C101F7
:101EE8008A014B228A0194250730BA004030B80095
:101EF8002030AA00AB01AE01AF010D308A01692084
:101F08000A308A01692042308A01692050308A01EA
:101F1800692053308A0169203D308A0169200430E4
:101F2800A9004408A4004508A5006830B000B10124
:101F38008A01A6200D308A0169200A308A016920A9
:101F48000730BA004030B8002030AA00AB01AE011B
:101F5800AF0153308A01692050308A01692043302B
:101F68008A0169203D308A0169200430A90083165E
:101F78005A088312A400A5016830B000B1018A0193
:101F8800A6200D308A0169200A308A0169200730AD
:101F9800BA004030B8002030AA00AB01AE01AF0152
:101FA80052308A01692053308A01692043308A01FE
:101FB80069203D308A0169200430A90083162C0865
:101FC8008312A40083162D088312A5006830B00080
:101FD800B1018A01A6200D308A0169200A308A01E0
:101FE80069200730BA004030B8002030AA00AB01A1
:101FF800AE01AF0152308A01692045308A0169205B
:1020080043308A0169203D308A0169200430A900E3
:10201800831624088312A400831625088312A500BA
:102028006830B000B1018A01A6200D308A0169200C
:102038000A308A0169200730BA004030B8002030E1
:10204800AA00AB01AE01AF0146308A0169204130D8
:102058008A01692054308A01692020308A01692068
:1020680073308A01692065308A01692063308A01EA
:10207800692073308A0169203D308A016920043063
:10208800A9007608A4007708A5006830B000B1015F
:102098008A01A6200D308A0169200A308A01692048
:1020A8000730BA004030B8002030AA00AB01AE01BA
:1020B800AF0154308A0169204F308A0169205330BA
:1020C8008A0169203D308A0169200430A9008316FD
:1020D80036088312A400831637088312A5006830D7
:1020E800B000B1018A01A6200430A900831638087F
:1020F8008312A400831639088312A5006830B00043
:10210800B1018A01A6200D308A0169200A308A01AE
:1021180069200730BA004030B8002030AA00AB016F
:10212800AE01AF0152308A01692044308A0169202A
:1021380053308A0169203D308A0169200430A900A2
:10214800831622088312A400831623088312A5008D
:102158006830B000B1018A01A6200D308A016920DB
:102168000A308A0169200730BA004030B8002030B0
:10217800AA00AB01AE01AF0146308A0169204430A4
:102188008A01692053308A0169203D308A0169201B
:102198000430A9007808A4007908A5006830B000C8
:1021A800B1018A01A6200D308A0169200A308A010E
:1021B80069200730BA004030B8002030AA00AB01CF
:1021C800AE01AF0146308A0169205F308A0169207B
:1021D8004F308A01692072308A01692069308A018A
:1021E800692067308A0169203D308A0169200430FE
:1021F800A9005408A4005508A5006830B000B10132
:102208008A01A6200430A9005608A4005708A50092
:102218006830B000B1018A01A6200D308A0169201A
:102228000A308A0169200730BA004030B8002030EF
:10223800AA00AB01AE01AF0146308A0169204130E6
:102248008A01692054308A01692031308A01692065
:102258005F308A01692061308A01692064308A010F
:10226800692064308A01692072308A0169203D3012
:102278008A0169200430A9005808A4005908A5005B
:102288006830B000B1018A01A6200430A9005A08BC
:10229800A4005B08A5006830B000B1018A01A6203F
:1022A8000D308A0169200A308A0169200730BA0096
:1022B8004030B8002030AA00AB01AE01AF01463073
:1022C8008A01692041308A01692054308A016920D5
:1022D80032308A0169205F308A01692061308A01C1
:1022E800692064308A01692064308A01692072306B
:1022F8008A0169203D308A0169200430A9006008FC
:10230800A4006108A5006830B000B1018A01A620C8
:102318000430A9006208A4006308A5006830B00072
:10232800B1018A01A6200D308A0169200A308A018C
:1023380069200730BA004030B8002030AA00AB014D
:10234800AE01AF0152308A0169206F308A016920DD
:102358006F308A01692074308A01692044308A010B
:10236800692069308A01692072308A0169205F30EA
:102378008A01692061308A01692064308A016920F4
:1023880064308A01692072308A0169203D308A01EF
:1023980069200430A900831628088312A400831634
:1023A80029088312A5006830B000B1018A01A6206F
:1023B8000430A90083162A088312A40083162B0868
:1023C8008312A5006830B000B1018A01A6200D3043
:1023D8008A0169200A308A0169200730BA00403032
:1023E800B8002030AA00AB01AE01AF0143308A012A
:1023F80069206C308A01692075308A016920733040
:102408008A01692074308A01692065308A0169204F
:1024180072308A0169205F308A01692073308A012D
:10242800692069308A0169207A308A01692065301B
:102438008A0169203D308A0169200430A9004808D2
:10244800A4004908A5006830B000B1018A01A6209F
:102458000D308A0169200A308A0169200730BA00E4
:102468004030B8002030AA00AB01AE01AF014230C5
:102478008A0169204F308A0169204F308A0169201A
:1024880054308A01692020308A0169204F308A013E
:1024980069204B308A0169200A308A0169200D3091
:1024A8008A0169208A150A1272200730BA00403062
:1024B800B8002030AA00AB01AE01AF0144308A0158
:1024C800692049308A01692052308A016920203008
:1024D8008A0169204F308A0169204B308A016920BE
:1024E8000A308A0169200D308A0169208A150A128A
:1024F80009230730BA004030B8002030AA00AB01E9
:10250800AE01AF0146308A01692041308A01692055
:1025180054308A01692020308A0169204F308A01AD
:1025280069204B308A0169200A308A0169200D3000
:102538008A0169208316AE01AF01831208008A154B
:102548000A126A270730BA004030B8002030AA00C3
:10255800AB01AE01AF0146308A01692041308A01E2
:10256800692054308A0169200230A9008316550871
:102578008312A400A5016830B000B1018A01B92016
:102588000A308A0169200D308A01692083162130BA
:10259800D2000130B200B3018312831632088312CD
:1025A800A000831633088312A100A30120308A01FA
:1025B80077218A110A16031D192B8316C601C70134
:1025C8008312831646088312A000831647088312D5
:1025D800A1000130A300FF308A0177218A110A1671
:1025E800031D022B8A150A1292238316C60A0319A1
:1025F800C70A8A110A168312031DE52A8316D20A0E
:1026080064007F3052028A110A168312031C102BB1
:1026180083162130D20083128316B20A0319B30A33
:102628008A110A168312031DD12A8A110A16882BC9
:102638000730BA004030B8002030AA00AB01AE0124
:10264800AF010A308A0169200D308A0169204130C2
:102658008A01692062308A0169206F308A01692005
:1026680072308A01692074308A01692065308A01D4
:10267800692064308A01692021308A0169200D307F
:102688008A0169200A308A01692046308A01692056
:1026980041308A01692054308A01692031308A0129
:1026A800692032308A01692020308A01692063302C
:1026B8008A01692061308A01692072308A016920A3
:1026C80064308A01692020308A01692064308A01D7
:1026D800692065308A01692074308A016920653073
:1026E8008A01692063308A01692074308A0169206F
:1026F80065308A01692064308A0169200D308A01B9
:1027080069200A308A0169200730BA004030B800D1
:102718002030AA00AB01AE01AF010A308A0169205E
:102728000D308A01692044308A0169204F308A01BE
:1027380069204E308A01692045308A01692021309C
:102748008A01692064008A110A16A62B63008A117F
:042758000A16AA2B88
:02400E003D3D36
:00000001FF
